:1000000026C1189518951895189518951895F8C043
:10001000189507C1189531303030313030300260DA
:1000200000000FEF07BB01E109B900E90AB900E2DE
:100030001EE401D100E824D008EC10E0FCD000EA76
:100040001FD008EC10E0F7D000E01AD000E80FBF96
:1000500000E00CB90CE001BB0CE002BB00E00FBFFC
:1000600000ED17E0E8D0E1E60081013031F4E0E690
:10007000008106D000E0E1E6008300E80FBFEECF8C
:1000800007D1C851502EA0E0B0E097E081E04424B1
:1000900066241C2F26E130E0012FE22FF32F48E0E9
:1000A000EED008E210E0C7D00CE001BB0CE002BBD0
:1000B00004E610E0C0D004E002BB04E610E0BBD0D0
:1000C00000E002BB442490E01DC0EC2FE40D6080F2
:1000D000439404E610E0AFD0062D000F000F000F90
:1000E00002BB04E610E0A7D0062D000F000F000FA2
:1000F000046002BB04E610E09ED0660C660C660C41
:1001000062BA9395983008F304E610E094D004E0C6
:1001100001BB00E002BB04E610E08DD081E004E00A
:1001200002BB04E610E087D081E002C080B3887093
:100130008823E1F700E002BB0CE001BB98E011C0AE
:10014000052D42E08ED0A42FB0E0052D42E089D0ED
:10015000502EEC2FE85F9A95092F000FE00FA08337
:10016000B183992369F7442490E023C0EC2FE85F22
:10017000042D000FE00FA081B18143940A2F08BB2A
:1001800004E610E058D00A2F000F000F000F02BB4A
:1001900004E610E050D00A2F000F000F000F04609B
:1001A00002BB04E610E047D0AA0FAA0FAA0FA2BB19
:1001B00093959830D8F204E610E03DD004E001BBFE
:1001C00000E002BB04E610E036D081E004E002BBB0
:1001D00004E610E030D081E002C080B3887088234C
:1001E000E1F700E002BB08E002BB08EC10E023D01E
:1001F0000CE002BB08EE13E01ED0C85EE7E050C082
:10020000EA931A930A9300E00AB90CB1E0E600837E
:10021000E0E6008118E41AB90CB909911991E99145
:100220001895EA930A9300E90AB901E0E1E6008330
:100230000991E991189531D080E090E080E090E05C
:1002400001C0019680179107E0F3E2E02EC001EAB9
:100250000DBFC2E831D0002309F03BD0E2DE57D019
:1002600056C00024E8E0EA9532F0001F001C041696
:10027000D0F3041AF8CF001F402D00950895AF93D6
:10028000A02FC89531960D924A95D9F7AF91089550
:100290006A925A924A92BA93AA939A938A93089529
:1002A0006E805D804C80BB81AA81998188810FB668
:1002B000F894CE0F0FBE089501E0089510E01D934D
:1002C0000A95E1F70895C89531960D920A95D9F7E8
:1002D00008958EE190E0E82FF92FC895002D319612
:1002E000C895A02DE82FF92F3296C895202D31966C
:1002F000C895122F102921F0E22FF02DE4DF01C064
:10030000DDDF049610E08232910728F308950000A3
:040310008895FECFFF
:00000001FF
